:030000000218F9EA
:0C18F90078FFE4F6D8FD7581C2020036CD
:0100110022CC
:061650008B308A31893263
:10165600756A027F48121776121951EF20E0F9AB2E
:1016660030AA31A9321206707872E6FE08E6FDED60
:01167600FF74
:011677002250
:100E910043525354005341564500434647002D3EAB
:100EA10053320052415445434C5220554E4954420D
:100EB1004C4E4B5452455644464C54534156455260
:100EC100535420535720202E3235203173202032A5
:100ED100732020357320203130732033307320315B
:100EE1006D2020326D2020356D202031306D203372
:100EF100306D203168202032682020346820205451
:100F01007269670000000100040008001400280055
:100F11007800F001E004B009601C2038407080E1E5
:100F210000FFFF46656574596172644D6574724FC7
:0F0F31006666204F6E20204E6F2020596573207A
:0C19050025E02404F582E4340FF5832271
:1014FB0078B576AB0876CD087600087604E408F666
:10150B0008760108F60876FA08764008F608F60819
:10151B00F608F67BFF7A0E79911215977F05121458
:04152B00900215FA1B
:10179100756E1D756FC01214C678B6E664CD7004FF
:0917A10018E664AB60031214FBAE
:0117AA00221C
:0D18C100C2AF7DC07C1DE4FF12184DD2AFF8
:0118CE0022F7
:1014C600753FFF856E40856F417542007543007517
:1014D60044B5E4FFAB3FAA40A9418F827583001251
:1014E6000643AB42AA43A9448F8275830012068243
:0414F6000FBF0EE036
:0114FA0022CF
:1015FA007D01E4FF12171E7BFF7A0E79961215976A
:10160A001218C1C2AF7FB57B0E7DC07C1D12185760
:0D161A00D2AF7F02121490E4FDFF02171EF4
:100A1A00E4F5307BFF7A0E799B1215977F05121445
:100A2A0090A297829650FAA296920FA2979210E5F8
:100A3A003075F004A424A4F9740E35F0FA7BFF1281
:100A4A0015977F05121490853031E4F5327BFF7AD1
:100A5A000E799F121597E53024FE602B146030142E
:100A6A006035240470397F01EF12190578B7E6FC66
:100A7A0008E6FD7401936D7003E4936C70028F3283
:100A8A000FBF10E4020B1D78B9E6F532020B42786B
:100A9A00BAE6F532020B5F78C1E6F532020B7CE565
:100AAA00306531708AA20F309601B35013A2969224
:100ABA000F30960C0530E530C394084003E4F53056
:100ACA00A210309701B350D7A29792103097D0E571
:100ADA0030B4080050C9900AE7F8282873020AFFC0
:100AEA00020B2A020B30020B4D020B6A020B900218
:100AFA000B96020B9C0532E532C394104003753203
:100B0A0001E532121905E493FF74019378B7CFF621
:100B1A0008EFF6E53275F004A424C4F9740E805B7C
:100B2A0012114E020AA90532E532C394034003E4C6
:100B3A00F53278B9A632E53275F004A42424F974A2
:100B4A000F80380532E532C394024003E4F5327867
:100B5A00BAA632E53275F004A42430F9740F801B6A
:100B6A000532E532C394024003E4F53278C1A63275
:100B7A00E53275F004A42438F9740F35F0FA7BFFD6
:100B8A00121597020AA91214FB020AA91215FA02EF
:080B9A000AA943A208020AA9FE
:0A191D004552415300444F4E45006F
:10173C00E4D3FCFD7B80FAF9F80207CF78B7E6F525
:0D174C005608E6F55722E563AE62780622E6
:10102F00C20DC20EE4F531F532AE31AF3212173CBC
:10103F00401CE53064816016AF32AE311215C91213
:10104F0018398F300532E53270DF053180DBE5303E
:10105F00B48108E532153270021531AE31AF32E48A
:10106F00C312173E700CD20D1218DDE4F562F56352
:10107F008007853162853263E4F564F565755580C7
:03108F00121748ED
:01109200223B
:0415C9008F828E83FC
:1015CD0012173C4027E582AE837806C333CE33CE67
:1015DD00D8F9FD756A02EE7872F6CFEDCFEF08F609
:0C15ED007F501217F7121951EF20E0F99F
:0115F90022CF
:0317AB00CDEFCDB2
:1017AE00756A02EE7872F6ED08F67F501217F71290
:0617BE001951EF20E0F9D3
:0117C4002202
:10183900756A017F50121776121951EF20E0F97875
:0318490072E6FF45
:01184C002279
:101824001217ABE4FFFE0FBF00010EBE0FF8BFA0FE
:04183400F512183958
:01183800228D
:06152F00CBEFCBCAEECAAF
:10153500300D03300E27756A03EA7872F6EB08F66C
:1015450008EDF67F501217F7121951EF20E0F9E474
:0D155500FFFE0FBF00010EBE0FF8BFA0F596
:011562002266
:10136000753300753400753555E4F532121752C3E4
:1013700033CE33CED8F97C002532FFEC3EFEAB33C2
:10138000AA34A935853282758300120643FD1215F1
:101390002F0532E532C3940640D2756400756506A8
:0113A000222A
:100F40008E308F31121752C333CE33CED8F9256588
:100F5000FFE5643EFEEEC0E0EFC0E0E530FDD0E02E
:100F6000FFD0E0FE12152F0565E5657002056412DD
:100F70001752C333CE33CED8F92565FFE5643EFE64
:100F8000AD3112152F0565E565700205640559E55B
:100F90005970020558C3E5659440E5649400401714
:100FA000E4F564F5650563E56370020562AE62FF12
:080FB00012173C5002D20D2281
:10114E00E4F564F5657BFF7A19791D121597D20EB9
:10115E00E4F53FF540AE3FAF4012173C4021E5406D
:10116E00AE3F7806C333CE33CED8F9F5658E647DA7
:10117E0081FF12152F0540E54070DA053F80D6C27B
:10118E000E7BFF7A197922121597E4F562F563F555
:05119E0064F565C20DBF
:0111A3002229
:1010F700E4F53FF540F541F542AE41AF4212173CEA
:101107004044E5406481603EAF42AE411215C912CA
:1011170018398F40E54064807022AF3F053FFCFDE2
:10112700FEFBFAF9120BA27F2C12000EAE41AF4262
:10113700E4FCFDFBFAF9120BA212193A0542E5424B
:0611470070B7054180B302
:01114D00227F
:021293008F3F8B
:10129500E4F540F541F542F543AE42AF4312173C44
:1012A5004030E5416481602AAF43AE421215C91250
:1012B50018398F41E541B4800FE540653F7007AFB0
:1012C50043AE420215C905400543E54370CB0542CF
:0212D50080C7D0
:0112D70022F4
:10180E00121748E4F558F559121360856266856320
:06181E00677F0102109338
:10145800856230856331E565456460080531E531AD
:101468007002053085666285676312136085306295
:10147800853163AE30AF3112173C5007E4F562F5A1
:0814880063D20D7F02021093F4
:10184D00740478FF769612FF0322740078FF769663
:04185D0012FF032251
:03003300020DCBF0
:0D0DCB00C0E0C0F0C083C082C0D075D00869
:100DD800E5D954F8FF1208480E05080E05100E1440
:100DE800180E2F200E16280E2F300E31380E3740D1
:100DF8000E2F480E50500E6D5800000E7B856DDA90
:100E0800C2DDC2DC756B00756C008070800EE56A0F
:100E180070028056056CE56C7002056B1200268F17
:100E2800DAC2DDC2DC80558016D2DDC2DC804DC25C
:100E3800DDC2DCE56A7004C2DA8041D2DA803DC2E4
:100E4800DDD2DC7568048034AFDA121911056CE55F
:100E58006C7002056BC2DDC2DCE56A7004C2DA8020
:100E68001BD2DA8017AFDA121911C2DDD2DC75682D
:0E0E7800028009756804C2DDC2DCD2DAC2DB7A
:0B0E8600D0D0D082D083D0F0D0E0327A
:1016270043910C43920CE4F5DBEF25E0F5DB300F3B
:101637000343DB0175DD2575DC2575D84453F8FEBA
:0916470053F7FEE4F568D2E82235
:1017F700E56830E002FF22E4F569756803EF25E04C
:07180700F56DD2DD7F022226
:10177600E56830E002FF22E4F569156A756805EF51
:0B17860025E04401F56DD2DD7F02225A
:0619510020DBFDAF68225F
:0D002600156AAF69056974722FF8E6FF22B4
:0C19110074722569F8EFF60569156A226A
:0E18CF00E4F5847585FFF592F5A475A5FF225A
:07194300EE3395E0FDFC22EC
:10167800C20AC20CC209D2A2C2A0C2A1E4FDFF12D2
:10168800171EE4FD7F0112171E7F081210937F04B6
:03169800021093AA
:10171E00EF146011047016BD0104C2A78002D2A797
:0E172E00A2A7920B22BD0103C2A622D2A622C0
:10109300EF14B40800505C9010A875F003A4C58346
:1010A30025F0C583730210C00210C60210CD0210D2
:1010B300D90210DB0210D90210E50210EDD20A7535
:1010C300190122C20AA20B92A722D20C751A057D1E
:1010D300017F0102171E8005C209C28722C209D2FD
:1010E3008722D209D28775180122C2A47F01121464
:0410F30090D2A422D1
:1013E000300A12D5190F30A707C2A775191E80053C
:1013F000D2A7751946E51AD39400400CD51A09C234
:101400000CE4FD7F0112171E300911D5180E30872C
:0D14100006C28775180522D28775181E22A6
:1016DE00C374039FFE1392A0EEA2E192A1AF80CF3E
:0F16EE005480CFED547FCF4FCF8F80C2A2D2A2B6
:0116FD0022CA
:061597008B418A428943EA
:10159D00E4FCCFECCF7D201216DE0CBC04F4E4FC91
:1015AD00AB41AA42A9438C82758300120643FD60AC
:0B15BD000ACFECCF1216DE0CBC04E5D8
:0115C8002200
:040FB8008F828E8313
:100FBC00121943E47B0F7A27F9F8C31207CF5003B9
:100FCC0090270FAF82AE831219437B197AFC79FFFD
:100FDC0078FFD31207CF400390FC19E4F530741B53
:100FEC002530F8E4F60530E530B405F2AE83AF8277
:100FFC001219437B007A00791B120BA2E51E701AA2
:10100C00753003741A2530F8E6FF741B2530F8C6CA
:10101C00EFC6D530EE751B2080E27B007A00791B81
:03102C0002159713
:1017C50046554C4C0050524F47005A4C4F47004D20
:0917D5004F44310076312E37003B
:030013000216BD15
:1016BD00C0E0C0D075D01020060CAF8DEFAD8BF50E
:1016CD005BEDF55CD206758D00758B00D0D0D0E04A
:0116DD0032DA
:021490008F408B
:10149200E4F541F542C3E5429540E541940050230D
:1014A200900000AF82AE83E4FCFD7B207A4EF9F817
:1014B200D31207CF4003A380EA0542E54270D60566
:0314C2004180D294
:0114C5002204
:0E18DD007BFF7A1779C51215977F0A021490C7
:100036001218CF1219271216787F041214902097DF
:10004600127BFF7A1779CA1215977F011212D8D23E
:10005600AF80FE2096091203BB12102F120A1A7ADD
:100066001779CF1203B07A1779D41203B07BFF7ACF
:100076001779D91215977F04121490E4FF1212D83B
:100086001203BB7F0112149012102F120011C2121C
:1000960012141D7F01121490E4F55DF55E12001234
:1000A600A2969200A2979201E4F52378A912082F4E
:1000B60000000000E4F52478B112082FFFFFD8F104
:1000C60078A512082F00000000E4F55478AD120858
:1000D6002F00000000C205C203C204E4F560F5610A
:1000E600F525F526F55BF55CC206F55FC20730120D
:1000F600FDC212300433A200309601B3400BA201B8
:10010600309701B340030201CD30961230970FC2EB
:1001160004E4F560F5617F04121093E4F554A296A9
:100126009200A29792010201CD209605209702D255
:100136000830964030973D30081BC20878B1120847
:100146002F0000000078AD12080A78A5120823D205
:1001560001D200802478BAE6601F0561E56170026D
:100166000560D394B8E560940B400ED2047F051267
:1001760010938005E4F560F561A200309601B35056
:100186001DA2969200309616200813E5546007E4E7
:10019600F5547F0680057554017F07121093A2015E
:1001A600309701B35021A297920130971A20081771
:1001B600B20330030F300D071218DDC20380081298
:1001C600180E80031214581203C820060302025E9A
:1001D600C2AFC206D2AFE4855C2F855B2EF52DF546
:1001E6002CAF2FAE2EAD2DAC2C7B107A27F9F81242
:1001F60006A48F2F8E2E8D2D8C2CE4FB7A90F9F889
:1002060012131C8F2F8E2E8D2D8C2C78C1E6600933
:10021600C374B89FFF740B9EFEE55F14601624FE40
:1002260060202403702FC3EF94B0EE9404500E7533
:100236005F018009D3EF9414EE9405401B755F03AC
:100246008016C3EF94B0EE9404500D755F01300331
:1002560007D2078003E4F55F0524E524C39405501F
:10026600030203AAE4F524FB7A0079271216508EBE
:10027600288F29E527640260030203AA78A91208D9
:1002860016E8C0E0E9C0E0EAC0E0EBC0E078B9E615
:10029600FDAF29AE28121247D0E0FBD0E0FAD0E03D
:1002A600F9D0E0F8EB2FFFEA3EFEE93DFDE83CFC25
:1002B60078A91208230523E523C3940550030203F6
:1002C600AA78A912080AE47B05FAF9F812131C7831
:1002D600A912082378A912080A78A5120816C3EFEE
:1002E6009BFFEE9AFEED99FDEC98FC78A912082387
:1002F60078B112080A78A9120816D31207CF400A55
:1003060078A912080A78B1120823E554600A78B36E
:10031600E6FE08E68E2AF52B78ABE6FE08E68E2882
:10032600F529E5546006AF2BAE2A8004AF29AE2826
:10033600120FB830035878B7E6FE08E6FFF47002ED
:10034600EEF460180526E52670020525C39FE5250F
:100356009E4010E4F525F526D2028007300704C238
:1003660007D202300228C2027F0312109330050D15
:10037600E528FF12000EAF29E52912000E200D090F
:10038600AF29AE28120F4080051218DDC20378A9E6
:1003960012080A78AD12082378A912082F00000067
:0A03A60000E4F5231213E00200F456
:1003B0007BFF1215977F0412149022D2AF1217916F
:0803C000C20F7F701216272204
:10169B00444C0021536967005A4C4F47004D4F444F
:1016AB003100312E37004D61722032332032303011
:0216BB003400F9
:1011F600AF38AE37AD36AC35EC4D4E4F22EF24FF4F
:10120600F538EE34FFF537ED34FFF536EC34FFF5FF
:101216003522E475382075374EF536F53522E475F6
:101226003801F537F536F53522FDFCAB38AA37A976
:1012360036A835C30207E57532007533007534B537
:011246002285
:1003C8001218EBEF70030205F37F04121093E4F5A3
:1003D80054C204F560F561121759EF12084805E791
:1003E8002405F02A054552040E61047C6304CF6598
:1003F800051A6C052072051D7305497405BC760540
:10040800B478000005F37BFF7A16799B12159712D2
:1004180012181218EBEF700A1211F6600512120387
:1004280080F01211F670030205F31217598F31127A
:100438001293E4F538121228E47F06FE12122F50A8
:100448000A1218398F311205F480ED1218398F31DC
:10045800E53164806016E5316481601012000E1287
:1004680018398F3112000E7530018003E4F530E53C
:100478003070D82212123D121224F5311211F66092
:10048800241212181218EBEF700A1211F6600512F6
:10049800120380F01211F6600312060D0531E531E2
:1004A800C3940E40D71211F6601A78B5B6AB070898
:1004B800B6CD030205ED7BFF7A16799E1215977F5C
:1004C8000A0214900205B1E4FFFE1217ABE4F538F6
:1004D800121228E4FF7E0812122F50331218398F97
:1004E80030E538540FFFE4FEFDFCFBFAF9F8C312BF
:1004F80007E5700F12193AAE37AF381218B07F20DF
:1005080012000EAF301217DE7F201205F480C402ED
:1005180005E4B205220210F712123DE4F531AB32C0
:100528000534E534AA337002053314F912062AFF9C
:1005380012000E0531E531C3940E40E22243A208B1
:1005480022753200753300753470121224F5311299
:1005580011F660241212181218EBEF700A1211F635
:10056800600512120380F01211F6600312060D05E1
:1005780031E531C3940240D71211F6602CAE70AF4A
:1005880071EE3395E0FDFC78AD120816C3EF9BF5CC
:100598003CEE9AF53BED99F53AEC98F539AF3C7895
:1005A800BFE53BF608EFF6803C0214C67F04121044
:1005B8009302114E7A1679A31206217A1679A81297
:1005C80006217F7612000E7BFF7A1679AD12189DF0
:1005D80012193A7BFF7A1679B112189D02193AE47A
:0B05E80078BFF608F60215FA1214FBAB
:1005F3002212000EE5382401F538E43537F537E4E7
:100603003536F536E43535F53522121759AB32AAAE
:1006130033A934853182758300EF120682227BFF72
:0706230012189D12193A2282
:0A192700E4F5955396BF53A27F220A
:10141D005389F0438901538FFE758C70E4F58A531F
:10142D00B8FD53B7FDD2A9D28C53890F4389905380
:10143D008FEFF58DF58B4391105392EF53B8F75312
:0B144D00B7F7D2ABD28ED28AD2AA220F
:03000B00021931A6
:09193100D212758C70758A003227
:03001B0002194A7D
:07194A00758D00758B003262
:101861000D0A00303132333435363738394142438D
:0418710044454600A4
:10187500AF53AB47AA48A949055322AF46AE45AD7C
:0418850044AC43220A
:1012D8005387BF75985053877FE4F5BABF0105431C
:1012E800A240800353A2BFE4F5BD75BE30F5BF75BB
:1012F800BD035391FE4392014391025392FDC213E1
:1013080053B8EF53B7EF43B81078A3F618F678A49C
:04131800F6D2AC223B
:0300230002156360
:10156300C0E0C0D075D01030981E78A3E6C3940FA6
:10157300501418E6062492F8A69978A30618E6C331
:10158300941040027600C298309904C299C213D0D5
:04159300D0D0E032A2
:080003002013FDD2138F992296
:1016FE0078A3E6D39400401508E6062492F8E6FF98
:0F170E0078A31608E6C394104005E4F6227F0086
:01171D0022A9
:03000E00020003EA
:101759007F207E4E78A3E67010D3EF9400EE9400BC
:0C1769004007EF1F70EE1E80EB1216FE12
:011775002251
:10189D0012062AFF600C12000E740129F9E43AFABF
:0318AD0080EE22A8
:0E18EB0078A3E6D3940040037F01227F002201
:1017DE00CEEFCEEE54F0C4540F90186493FF120067
:0917EE000EEE540F93FF02000EF1
:1018B000CDEFCDCCEECCEEFF1217DECFEDCF021781
:0118C000DE49
:09193A007BFF7A18796102189D07
:0E0BA2008F468E458D448C438B478A48894987
:100BB000E4F553EC4D4E4F7017E94A4B70057F300A
:100BC00002000E1218758F827583007430020CC5F6
:100BD000121882EC33502AE5494548454770077F93
:100BE0002D12000E800D1218758F82758300742DE2
:100BF0001206821218801207C18F468E458D448CD2
:100C000043755201754D00754CCA754B9A754A3B38
:100C1000E4FFFEFDFCAB4DAA4CA94BA84AD312073A
:100C2000E55003020CB0121880A84A12072F8F510A
:100C30008E508D4F8C4EEC4D4E4F7004E55270230C
:100C4000E5512430FFE54945484547700512000E3F
:100C5000800EAE531218778E82758300EF120682D3
:100C6000E4F552AF4DAE4CAD4BAC4AAB51AA50A9D6
:100C70004FA84E1206A4C8ECC8C9EDC9CAEECAC333
:100C8000E5469FF546E5459AF545E54499F544E581
:100C90004398F543AF4DAE4CAD4BAC4AE47B0AFAFA
:100CA000F9F812072F8F4D8E4C8D4B8C4A020C1089
:100CB000E548454945476010AB47AA48A9498553CF
:080CC00082758300E412068234
:010CC8002209
:10086E000134C35001DBBF68028BBB800344B798D1
:10087E000407B3B004D5AFC805A9ABE00689A7F845
:10088E000775A410086DA02809719C400A8198581C
:10089E000B9F94700CCA90880DE98CF90E048CA0F5
:1008AE000EA88AAC0F4D88B80FF786C410A184D05D
:1008BE00115182DC120580E812BB7EF413747D00A8
:1008CE0014307B0C14F2791815B877241680753015
:1008DE00174B733C1819714818ED6F5419C46D609D
:1008EE001AA16B6C1B7E69781C6167841D4A65902A
:1008FE001E37639C1F2561A8201A5FB421125DC0AC
:10090E00220D5BCC230E59D8241557E4251F55F024
:10091E00262F53FC27425208285B501429764E206E
:10092E002A9B4C2C2BC04A382CEE48442E1E465087
:10093E002F55445C308F426831D1407433173E805E
:10094E0034633C8C35B13A98370938A4386636B0E2
:10095E0039C734BC3B2D32C83C9D30D43E0F2EE0FF
:10096E003F882CEC41062AF8428D290444182710A2
:10097E0045AB251C4741232848E121344A861F40B8
:10098E004C311D4C4DE21B584F9C1964515D177034
:10099E005323157C54EF138856C4119458A20FA0FC
:1009AE005A830DAC5C6D0BB85E6009C4605807D0FD
:1009BE00625A05DC646203E8667301F4688A00001B
:1009CE006AA1FE0C6CB8FC186ECFFA2470E6F830F3
:1009DE000000000000000000000000000000000009
:1009EE0000000000000000000000000000000000F9
:1009FE0000000000000000000000000000000000E9
:0C0A0E00000000000000000000000000DC
:1013A10075F004E537A4246EF582E5F03408F58381
:1013B100E49322FE740193FF75F004E537A422F54E
:1013C10083C37401939FFFE4939EFEE4228F388EC2
:0F13D100378D368C35228F348E338D328C31220E
:10188900C3EF9DEE9C400AD3EF9BEE9A50037F0174
:04189900227F002288
:040CC9008E358F369F
:100CCD00E4F5371213A1FC740193FD1213B92472CC
:100CDD00F582E5F03408F583E493FA740193FBAFE4
:100CED0036AE35121889EF7003020DB91213A11229
:100CFD0013B42472F582E5F034081213C08F3B8EC5
:100D0D003AF539F5381213B92474F582E5F0340843
:100D1D00F583E4931213B42470F582E5F0340812D0
:100D2D0013C08F3F8E3EF53DF53CAD3DAC3C1207FB
:100D3D00C18F3F8E3E8D3D8C3CAE35AF36E4FCFD14
:100D4D00EEC0E0EFC0E01213A1FE740193FBCAEEFA
:100D5D00CAD0E0FFD0E0FEC3EF9BFFEE9AFEED940C
:100D6D0000FDEC9400FCAB3FAA3EA93DA83C120649
:100D7D00A4AB3BAA3AA939A83812131CC8ECC8C9B0
:100D8D00EDC9CAEECACBEFCB1213B92470F582E5CB
:100D9D00F03408F583E493FE740193FFE4FCFDEB5E
:100DAD002FFFEA3EFEED39FDEC38FC220537E53725
:0D0DBD00C3946A5003020CD0E4FFFEFDFC5D
:010DCA002206
:0100120022CB
:1011A4001213CEAB38AA37A936A835E8C0E078BD0B
:1011B400E6FE08E6FFE4FCFDD0E0F81206A41213F4
:1011C400CE780E1207F61213CE78BFE6FE08E6FFBD
:1011D400EE3395E0FDFCE5382FF538E5373EF5377D
:1011E400E5363DF536E5353CF535AF38AE37AD3649
:0211F400FC22DB
:021247008D30E8
:10124900120CC91213D71211A41213D7E530146066
:101259001C14702DE47FE87E03FDFCAB34AA33A98E
:1012690032A8311206A4E47BE87A0B800CAF34AEC5
:1012790033AD32AC31E47B03FAF9F812131C1213C3
:09128900D7AF34AE33AD32AC3105
:011292002239
:10062A00BB010689828A83E0225002E722BBFE02CE
:09063A00E32289828A83E4932201
:10064300BB010CE58229F582E5833AF583E022506C
:1006530006E92582F8E622BBFE06E92582F8E222B6
:0D066300E58229F582E5833AF583E49322D0
:10067000BB010689828A83F0225002F722BBFE0169
:02068000F32263
:10068200F8BB010DE58229F582E5833AF583E8F0AE
:10069200225006E92582C8F622BBFE05E92582C85A
:0206A200F22242
:1006A400E88FF0A4CC8BF0A42CFCE98EF0A42CFCF5
:1006B4008AF0EDA42CFCEA8EF0A4CDA8F08BF0A473
:1006C4002DCC3825F0FDE98FF0A42CCD35F0FCEBD2
:1006D4008EF0A4FEA9F0EB8FF0A4CFC5F02ECD3997
:0F06E400FEE43CFCEAA42DCE35F0FDE43CFC2204
:1006F30075F008758200EF2FFFEE33FECD33CDCCBE
:1007030033CCC58233C5829BED9AEC99E582984040
:100713000CF582EE9BFEED9AFDEC99FC0FD5F0D61D
:10072300E4CEFBE4CDFAE4CCF9A88222B800C1B947
:100733000059BA002DEC8BF084CFCECDFCE5F0CB85
:10074300F97818EF2FFFEE33FEED33FDEC33FCEBBE
:1007530033FB10D703994004EB99FB0FD8E5E4F979
:10076300FA227818EF2FFFEE33FEED33FDEC33FC66
:10077300C933C910D7059BE99A4007EC9BFCE99A5A
:10078300F90FD8E0E4C9FAE4CCFB2275F010EF2F9F
:10079300FFEE33FEED33FDCC33CCC833C810D7079F
:1007A3009BEC9AE899400AED9BFDEC9AFCE899F8DA
:0E07B3000FD5F0DAE4CDFBE4CCFAE4C8F9226D
:10131C00C2D5E830E70FB2D5E4C39BFBE49AFAE4FC
:10132C0099F9E498F8EC30E717B2D512135212077A
:10133C002FE4C39BFBE49AFAE499F9E498F8800350
:10134C0012072F30D50DE4C39FFFE49EFEE49DFDF4
:04135C00E49CFC22EF
:0E07C100C3E49FFFE49EFEE49DFDE49CFC2249
:1007CF00EB9FF5F0EA9E42F0E99D42F0EC6480C8A1
:0607DF0064809845F02241
:1007E500EB9FF5F0EA9E42F0E99D42F0E89C45F06A
:0107F50022E1
:1007F600E86010ECA2E713FCED13FDEE13FEEF1319
:04080600FFD8F02205
:0C080A00E6FC08E6FD08E6FE08E6FF221A
:0D081600E6FB08E6F908E6FA08E6CBF82252
:0C082300ECF608EDF608EEF608EFF62201
:10082F00D083D082E493F608740193F60874029390
:09083F00F608740393F6740473C7
:10084800D083D082F8E4937012740193700DA3A33F
:1008580093F8740193F5828883E473740293686053
:06086800EFA3A3A380DF53
:00000001FF
